:020000040000FA
:0400000068303A2802
:08000800A000030EA100831209
:1000100081018B100B11210E8300A00E200E090010
:0C007400203084008001840A6030040207
:10008000031C3C281230B00033218316FF2390005C
:10009000831283160C308505870183128501870141
:1000A000073099000030831691009F008312C830FA
:1000B00083168100831231309000003083168C004B
:1000C000831210308B00831600309B001C141A081A
:1000D0008312BC00851D55213C1C762883161030E8
:1000E0009B001C141A088312BD003F2181018E0160
:1000F0008F010B118B100B108C018B179220311973
:1001000094201721B30B9028031085190314B90DFF
:10011000F0303902031951210F30390203194D21F2
:100120007B217E2864000800080031110130B700EF
:100130008B132030370783169B001C141A08831278
:10014000A4001030370783169B001C141A08831272
:10015000A3000030370783169B001C141A08831273
:10016000A2008B17321CBA2822090339A200A30966
:10017000A409A50901303702031DC3283D18C3286F
:100180003D143E14342101303702031DCC283D1CA0
:10019000CC283D103E143721CD28B70A0230370253
:1001A0000318080098280130B600B300B400B50069
:1001B000B70085018701B1139220B30BEF2803101C
:1001C00085190314B90DF030390203190D29B40B48
:1001D000EF280130370203193B219630B400311D5E
:1001E000DC283111321CF9282D090339AD00AE0984
:1001F000AF098B1320303707BB002F08BA0020212E
:1002000010303707BB002E08BA0020210030370716
:10021000BB002D08BA0020218B1785018701B70A82
:10022000B60102303702031CDC283F2108003E1CC7
:1002300008003E101030BB003D08BA002021080025
:100240008B133A0883161C159A003B089B00553007
:100250009D00AA309D009C1464009C182C291C1140
:1002600083128B17080008000130BD0008008701C9
:100270000530D40008000508333A85000800BD01A8
:100280003D14080001303D020319472908000130E0
:10029000D40056150730D30008003D143E14342115
:1002A00008003D103E1437210800B601B301B40127
:1002B0003C1C5D29BC01BC145F29BC013C143C08FA
:1002C000B6006400632964296529662967293330EB
:1002D000B41B8500B41F8501B30B6129B40B6129E0
:1002E0000310B60CB608031D61290030BB003C08A2
:1002F000BA00202108008F08031908008E018F0121
:10030000D0080319CB29D00F982956180516D618EE
:10031000851656190514D6198514D60158180512D4
:10032000D818851258190510D8198510D801CB296D
:100330005008D10056180516D618851656190514FA
:10034000D619851451080E020318B229581805123F
:10035000D818851258190510D8198510FF30500289
:10036000031908008F08031D0800922051080E028F
:10037000031CB22956180512D618851256190510F5
:10038000D619851058180516D81885165819051449
:10039000D8198514080000305302031DE4293D18C4
:1003A000DC29051A58140130051AD000851AD81412
:1003B0000130851AD00008000130D40056140130F5
:1003C000D0000130D3000800051AEA295614851A16
:1003D000D814EC29D61458140130D000D40B0800DE
:1003E00001305302031DFE29D6150530D40002301A
:1003F000D3003D180800D601D30108000230530293
:10040000031D102A56158714D8150330D400033065
:10041000D3003D1808008701D601D301D815080084
:1004200003305302031D202A871407150330D4001C
:100430000430D3003D1808008701D3015815080087
:1004400004305302031D312A8714071507140330A3
:10045000D4000530D3003D1808008701D30158159A
:10046000080005305302031D432A8714071507149B
:1004700087160330D4000630D3003D1808008701EA
:10048000D3015815080006305302031D562A87145D
:1004900007150714871607160330D4000730D3005A
:1004A0003D1808008701D301581508000730530292
:1004B000031D6A2A87140715071487160716871560
:1004C0000130D4000730D3003D1808008701D30164
:0A04D000581508000030D3000800A2
:084000000700030004000800A2
:02400E00CC01E3
:10420000FF00FF00FF00FF00FF00FF00FF00FF00B6
:10421000FF00FF00FF00FF00FF00FF00FF00FF00A6
:104220000100FF00FF00FF00FF00FF00FF00FF0094
:10423000FF00FF00FF00FF00FF00FF00FF00FF0086
:104240001000FF00FF00FF00FF00FF00FF00FF0065
:10425000FF00FF00FF00FF00FF00FF00FF00050060
:10426000FF00FF00FF00FF00FF00FF00FF00FF0056
:10427000FF00FF00FF00FF00FF00FF00FF00FF0046
:10428000FF00FF00FF00FF00FF00FF00FF00FF0036
:10429000FF00FF00FF00FF00FF00FF00FF00FF0026
:1042A000FF00FF00FF00FF00FF00FF00FF00FF0016
:1042B000FF00FF00FF00FF00FF00FF00FF00FF0006
:1042C000FF00FF00FF00FF00FF00FF00FF00FF00F6
:1042D000FF00FF00FF00FF00FF00FF00FF00FF00E6
:1042E000FF00FF00FF00FF00FF00FF00FF00FF00D6
:1042F000FF00FF00FF00FF00FF00FF00FF000000C5
:00000001FF
